:020000020000FC
:1000000014C07FC010C00FC00EC00DC06AC00BC0AE
:100010000AC009C008C007C006C005C004C003C0AC
:1000200002C001C000C0FFCF18958FED8DBF3324F3
:100030008FEF87BB38BA87E882BB8BBB809581BBCB
:100040003ABA30BE81E083BF82E089BF81E285BFDA
:1000500080E48BBF8FE0D82E7894112780B214D023
:1000600007FD04D005FD09D08895FACF0F77CD1490
:1000700011F4949A0895949808950F7DEB2DFF271D
:10008000EF73E859FE4F1491882D837099B391FB5B
:1000900082F990FB83F9C82E15FF03C01F70D12E83
:1000A00019C0DC14B9F414FF15C01A3121F438BAA0
:1000B0009598969814C0E8EAF1E01F70E10FF31DDF
:1000C000E10FF31D859198B3982798BB859192B362
:1000D000982792BB11279498CD1409F4949A11276C
:1000E00008952FB6739409F40068791441F4672CCD
:1000F000A2E3A60DA6BFA0EE4A2EAFEF5A2E2FBE4A
:1001000018952FB680B282FC02C0939AF8CF9398CC
:10011000A72DA619672C92E3972C990EA13138F3DD
:10012000A73110F4889405C0AB3108F3A132F8F67A
:100130000894441C551C57FCE2CF440C551C440C3D
:10014000551C4694469453FA46F8A7E05A22A7E075
:100150005A1609F0CCCF4B1419F04A1411F0A42C04
:10016000C6CFB42C0062C3CF0000000024252100BC
:1001700000000000000000262E000000000000002B
:10018000002D28292C202B2F1415181912131011AB
:100190001617161700000000001A00002A000000C1
:1001A00027000000000022230100020004000800D4
:0C01B000100020004000800000200040F3
:00000001FF
